:020000040000FA
:100000000C94FE000C9426010C9426010C942601FD
:100010000C9426010C9426010C9426010C942601C4
:100020000C9426010C9426010C9426010C942601B4
:100030000C9426010C9426010C9426010C942601A4
:100040000C94420F0C9426010C94B20F0C948C0F5C
:100050000C9426010C9426010C9426010C94260184
:100060000C94E40F0C94260100407A10F35A00A07F
:10007000724E18090010A5D4E80000E87648170071
:1000800000E40B54020000CA9A3B000000E1F505B1
:10009000000080969800000040420F000000A086FB
:1000A00001000000102700000000E803000000002D
:1000B0006400000000000A000000000001000000D1
:1000C00000002C76D888DC674F0823DFC1DFAE59EB
:1000D000E1B1B796E5E3E453C63AE651997696E87E
:1000E000E6C28426EB898C9B62ED407C6FFCEFBC02
:1000F0009C9F40F2BAA56FA5F490055A2AF75C932D
:100100006B6CF9676DC11BFCE0E40D47FEF520E662
:10011000B500D0ED902E0300943577050080841E45
:10012000080000204E0A000000C80C333333330FA0
:10013000986E12831141EF8D2114893BE65516CF3D
:10014000FEE6DB18D1844B381BF77C1D901DA4BB49
:10015000E424203284725E228100C9F124ECA1E5FE
:100160003D27CDCCCC3D0AD7233C17B7D13877CC2F
:100170002B329595E6241FB14F0A0000803FCDCC6D
:10018000CC3D6F12833A95BFD6337D1D9026B3CEFA
:10019000010C000020410000C84200401C4620BC69
:1001A000BE4CCA1B0E5AAEC59D740000000800026A
:1001B0000100000304070000000000000000000030
:1001C0000000250028002B0000000000240027006C
:1001D0002A000404040404040404020202020202C9
:1001E00003030303030301020408102040800102FB
:1001F00004081020010204081020031111241FBE5E
:10020000CFEFD8E0DEBFCDBF24E0ACE1B2E001C06B
:100210001D92AB31B207E1F712E0A0E0B1E0ECEBE8
:10022000FAE302C005900D92AC31B107D9F710E0A6
:10023000CEEFD0E004C02197FE010E945B1BCD3FB2
:10024000D107C9F70E9486110C945C1D0C94000024
:1002500091E09093BB028093DD021092BC02109259
:10026000DE0208950895089590E0FC01EA51FE4FE2
:1002700024918E529E4FFC018491882399F090E046
:10028000880F991FFC01E853FE4FA591B491FC0122
:10029000E254FE4F859194918FB7F894EC91E22B44
:1002A000EC938FBF089590E0FC01E655FE4F24913A
:1002B000FC01EA51FE4F3491FC01EE52FE4FE491F5
:1002C000EE23C9F0222339F0233001F1A8F42130C4
:1002D00019F1223029F1F0E0EE0FFF1FE254FE4F3A
:1002E000A591B4918FB7F894EC91611126C0309527
:1002F0003E233C938FBF08952730A9F02830C9F0E2
:10030000243049F7809180008F7D03C08091800068
:100310008F7780938000DFCF84B58F7784BDDBCF6C
:1003200084B58F7DFBCF8091B0008F778093B00034
:10033000D2CF8091B0008F7DF9CF3E2BDACF3FB77F
:10034000F8948091650290916602A0916702B09145
:10035000680226B5A89B05C02F3F19F00196A11D84
:10036000B11D3FBFBA2FA92F982F8827BC01CD01FF
:10037000620F711D811D911D42E0660F771F881F5E
:10038000991F4A95D1F708958F929F92AF92BF928D
:10039000CF92DF92EF92FF926B017C010E949F014E
:1003A0004B015C01C114D104E104F104B9F00E94D5
:1003B0009F01681979098A099B09683E7340810584
:1003C000910580F321E0C21AD108E108F10888EE16
:1003D000880E83E0981EA11CB11CE4CFFF90EF9023
:1003E000DF90CF90BF90AF909F908F900895AF9285
:1003F000BF92CF92DF92EF92FF920F931F93CF9312
:10040000DF936C017B018B01040F151FEB015E0173
:10041000AE18BF08C017D10759F06991D601ED9108
:10042000FC910190F081E02DC6010995892B79F7A7
:10043000C501DF91CF911F910F91FF90EF90DF9059
:10044000CF90BF90AF900895FC01448155816081A9
:1004500071818BE094E00C94F701FC01538D448D85
:10046000252F30E0842F90E0821B930B541710F05F
:10047000CF96089501970895FC01918D828D98176C
:1004800061F0A28DAE0FBF2FB11D5D968C91928D44
:100490009F5F9F73928F90E008958FEF9FEF089575
:1004A000FC01918D828D981731F0828DE80FF11D3E
:1004B000858D90E008958FEF9FEF0895FC01918D59
:1004C000228D892F90E0805C9F4F821B91098F7352
:1004D000992708958FED92E00E945E0221E0892B1A
:1004E00009F420E0822F089580E090E0892B29F024
:1004F0000E946A0281110C9400000895FC01A48DF1
:10050000A80FB92FB11DA35ABF4F2C91848D90E035
:1005100001968F739927848FA689B7892C93A08918
:10052000B1898C91837080648C93938D848D9813A2
:1005300006C00288F389E02D80818F7D8083089535
:10054000EF92FF920F931F93CF93DF93EC0181E023
:10055000888F9B8D8C8D98131AC0E889F9898081CA
:1005600085FF15C09FB7F894EE89FF896083E889FD
:10057000F98980818370806480839FBF81E090E0EF
:10058000DF91CF911F910F91FF90EF900895F62E7C
:100590000B8D10E00F5F1F4F0F731127E02E8C8D16
:1005A0008E110CC00FB607FCFACFE889F98980815B
:1005B00085FFF5CFCE010E947E02F1CFEB8DEC0FCF
:1005C000FD2FF11DE35AFF4FF0829FB7F8940B8F78
:1005D000EA89FB8980818062CFCFCF93DF93EC01E2
:1005E000888D8823B9F0AA89BB89E889F9898C911B
:1005F00085FD03C0808186FD0DC00FB607FCF7CFD7
:100600008C9185FFF2CF808185FFEDCFCE010E94D6
:100610007E02E9CFDF91CF910895089520913D02A8
:10062000260F3327331F21323105ECF42091B50218
:10063000FC0190E080E0243069F082E00895A09110
:100640003D022191AC01435E5D4FA40FB52FB11D5A
:100650002C930196861798F380913D02680F609362
:100660003D0280E0089581E008951092B50281E096
:100670008093B40210928F0261E082E10E945301E4
:1006800061E083E10E945301E9EBF0E080818E7F1D
:10069000808380818D7F808388E48093B80085E4A7
:1006A0008093BC00089510928E0210928D021092D9
:1006B000BC021092DE020E94350382E391E0909327
:1006C0008C0280938B0283E391E090938A02809363
:1006D00089020895CF93DF9391E090931C028823C1
:1006E000B9F0C091B800D091BA008091BC008A7B6B
:1006F0008093BC0060E082E10E94530160E083E1EE
:100700000E9453010E943503D093BA00C093B800F1
:10071000DF91CF910895CF92DF92EF92FF920F93E6
:100720001F93CF93DF93D091DE0281E0D13208F0A6
:100730009CC0C091DD020E949F016B017C018091F1
:10074000B50281116CC082E08093B50281E0809394
:10075000B4028FEF8093B3021092B202D093B10231
:10076000ADEBB2E0E1E9F2E080E0D8138DC0109289
:10077000900280919002CC0FC82BC0939002809180
:100780008F02813009F084C010928F020E949F0175
:100790006B017C01809190028093BB008091B70235
:1007A0009091B802A091B902B091BA02892B8A2B1C
:1007B0008B2BA1F00E949F010091B7021091B8020B
:1007C0002091B9023091BA026C197D098E099F09F6
:1007D000061717072807390708F442C08091BC00A4
:1007E00083FDD8CF85EC8093BC000E949F016B01F4
:1007F0007C018091B502823009F44CC08091B30233
:100800008F3F09F469C08091B302803209F466C059
:100810008091B302803309F463C084E026C08091E4
:10082000B7029091B802A091B902B091BA02892B97
:100830008A2B8B2B09F483CF0E949F010091B70272
:100840001091B8022091B9023091BA026C197D0959
:100850008E099F09061717072807390708F06FCF79
:100860008091B6020E946A0385E01092BC02109249
:10087000DE021092BB02DF91CF911F910F91FF908A
:10088000EF90DF90CF9008959D9191938F5F6DCF02
:1008900085EEA9CF8091B7029091B802A091B902DC
:1008A000B091BA02892B8A2B8B2B09F4A2CF0E941C
:1008B0009F010091B7021091B8022091B9023091C6
:1008C000BA026C197D098E099F09061717072807B8
:1008D000390708F08ECFC4CF80E0C7CF82E0C5CF04
:1008E00083E0C3CF0895E0918E0280918D02E817D6
:1008F00030F4F0E0E759FD4F808190E008958FEFEC
:100900009FEF089590918E0280918D022FEF3FEF1F
:10091000981748F4E92FF0E0E759FD4F208130E0C7
:100920009F5F90938E02C901089580918D029091EE
:100930008E02891B990B0895CF92DF92EF92FF925E
:100940000F931F93CF93DF937C01CB018A012091FA
:10095000BB02222389F0EB016B01C40ED51ECC151E
:10096000DD0569F06991D701ED91FC910190F0816D
:10097000E02DC7010995F3CF642F0E940E03C80133
:10098000DF91CF911F910F91FF90EF90DF90CF906B
:100990000895CF93DF931F92CDB7DEB7698320917F
:1009A000BB022223F9F02091DE02203258F021E030
:1009B00030E0FC013383228390E080E00F90DF91F0
:1009C000CF9108958091BC02E82FF0E0E354FD4FF1
:1009D000998190838F5F8093BC028093DE0281E0D7
:1009E00090E0ECCF61E0CE0101960E940E03F7CFBC
:1009F0000F931F93CF938C01C62FFC0184810E941B
:100A00002801F80163856C2B8CE793E00E94C904F0
:100A1000CF911F910F910C948B0390E080E008958B
:100A2000CF93DF93EC0188819981DC01ED91FC91FA
:100A30000190F081E02D09952A813B81820F931F5F
:100A40009B838A83DF91CF910895CF93DF93EC014D
:100A500088819981DC01ED91FC910280F381E02D88
:100A600009952A813B81820F931F9B838A83DF91A3
:100A7000CF9108958F929F92AF92BF92CF92DF92C3
:100A8000EF92FF920F931F93CF93DF93CDB7DEB713
:100A900066970FB6F894DEBF0FBECDBF6C018E0116
:100AA000095E1F4F78018AE0882E912CA12CB12C71
:100AB000CB01BA01A50194010E945F1A942F852FE2
:100AC000605DF80162938F01A901692F782F4115AC
:100AD00051056105710561F7A7014E1B5F0BBF0151
:100AE000C6010E94250566960FB6F894DEBF0FBEBC
:100AF000CDBFDF91CF911F910F91FF90EF90DF90CD
:100B0000CF90BF90AF909F908F900895FC0125816A
:100B1000222339F0F8E02F0290011124820F931F55
:100B2000089590E080E00895FB0101900020E9F72E
:100B30003197AF01461B570BDC01ED91FC91028010
:100B4000F381E02D0994FB0101900020E9F7319732
:100B5000AF01461B570B0C9425051F93CF93DF93D2
:100B6000E2E8F1E01281112379F0329621816213DB
:100B7000F9CFEC016CE50E941005612FCE01DF91E9
:100B8000CF911F910C9410056111F9CF63E971E0C9
:100B9000DF91CF911F910C94A3052F923F924F921A
:100BA0005F926F927F928F929F92AF92BF92CF92FD
:100BB000DF92EF92FF920F931F93CF93DF93CDB706
:100BC000DEB76C970FB6F894DEBF0FBECDBF8C01B9
:100BD0001B01DC0114968C9114978F77863009F4F1
:100BE00092C268F58230A0F11296ED90FC901397B6
:100BF000CC901196DC90843008F056C2A701B60163
:100C0000C1010E942505F101828193816C960FB686
:100C1000F894DEBF0FBECDBFDF91CF911F910F9132
:100C2000FF90EF90DF90CF90BF90AF909F908F900C
:100C30007F906F905F904F903F902F9008958C30F1
:100C400069F160F4883009F459C28A3009F43FC26E
:100C50006AE971E0C1010E94A305E5C1803209F48F
:100C6000ECC18034A9F76BE5C1010E941005F801C1
:100C7000008111810115110509F4DAC1B101C80122
:100C80000E94CD05C8010E9486058C01892B09F4BC
:100C9000CFC16CE2C1010E941005ECCFF801C08009
:100CA000D180E280F380A7019601C701B6010E94BE
:100CB0007A178111CDCF20E030E0A901C701B6013C
:100CC0000E947A17882379F0A7019601C701B6011F
:100CD0000E94E5189B01AC01C701B6010E947A177A
:100CE000882309F4B5CF20E030E0A901C701B6019F
:100CF0000E947A1787FF08C06DE2C1010E941005AB
:100D0000F7FAF094F7F8F09420E836E948E15BE46C
:100D1000C701B6010E94461A87FD81C074E1A72E63
:100D2000B12C00E210E0188E1F8AF501EE56FE4F3E
:100D30002591359145915491C701B6010E94461AFB
:100D400087FD13C0F501EE59FE4F25913591459170
:100D50005491C701B6010E94E0176B017C012F89F5
:100D6000388D200F311F388F2F8B1595079534E064
:100D7000A31AB1088CEFA8168FEFB806B1F6552468
:100D80005A9420E030E0A901C701B6010E94461A3A
:100D900018160CF04BC02CEA35EC47E257E3C701BC
:100DA000B6010E947A1718160CF440C0A52DB4E0C5
:100DB000AB02C0011124B12CA12CFC01E658FE4F5E
:100DC0003F019C012E563E4F49013FEF531671F1F2
:100DD000F301EA0DFB1D2591359145915491C70111
:100DE000B6010E947A1787FF13C0F401EA0DFB1DBC
:100DF0002591359145915491C701B6010E94E017A4
:100E00006B017C018F89988D801B910B988F8F8B44
:100E1000159507955A9494E0A91AB108D6CF00E227
:100E200010E055E0552E188E1F8AABCFC701B601D2
:100E30000E94C3194B015C012B013C0106E080E4D8
:100E400092E4AFE0B0E0898F9A8FAB8FBC8F102F08
:100E500001509AE04916510461047104C8F0698D8B
:100E60007A8D8B8D9C8D2AE030E040E050E00E942E
:100E70005F1A298F3A8F4B8F5C8FC301B2012AE032
:100E800030E040E050E00E945F1A29013A01DFCFD4
:100E9000C501B4010E947F179B01AC01C701B601D7
:100EA0000E94E4186B017C01698D7A8D8B8D9C8D7D
:100EB0000E947F179B01AC01C701B6010E94E01799
:100EC0002B013C010E94C3196B017C010E947F171A
:100ED0009B01AC01C301B2010E94E4189B01AC016B
:100EE0000E94E5180E94C319C60ED71EE81EF91EFF
:100EF000898D9A8DAB8DBC8DC816D906EA06FB0686
:100F0000D8F09FEF891A990AA90AB90AAF89B88D52
:100F1000AB2B39F1BAE08B169104A104B10408F1AE
:100F2000EF89F88D3196F88FEF8BC12CD12C76019B
:100F3000812C912C540183942AE0422E512C612C57
:100F4000712CC701B601A30192010E945F1A672BA1
:100F5000682B692B51F4111644F469017A01115080
:100F6000F0CFC12CD12C7601E7CFB501A401C1018E
:100F70000E943A05112371F14E01F1E18F0E911C8F
:100F8000012F54019AE0492E512C612C712C0150F3
:100F900068F0C701B601A30192010E945F1A605D6B
:100FA000D4016E934D0169017A01F1CF812F90E058
:100FB000BC0160957095F501E81BF90B31978EE245
:100FC000808344275527461B570B6A0D7B1DC101A3
:100FD0000E942505EF89F88DEF2B29F165E6C10107
:100FE0000E9410050F89188D17FF07C06DE2C1011F
:100FF0000E941005119501951109FE0177969F0138
:101000008AE0E82EF12CC801B7010E944B1A805DDE
:1010100082938B01672BB9F7A9014E1B5F0BBF01B0
:10102000C1010E942505D10112968D919C91EECDB2
:101030006DE5C1010E941005F6CF6BE7C1010E946A
:101040001005F801008111810115110559F1D80130
:101050001696CC9016971796DC9062E2C1010E941A
:1010600010057601F70161917F01662321F0C1012E
:101070000E94AD05F7CF62E2C1010E9410056AE34C
:10108000C1010E941005B101C8010E94CD05C8012F
:101090000E9486058C01892B29F06CE2C1010E9417
:1010A0001005D2CF6DE7C5CF62E2C1010E941005E5
:1010B0008601E00EF11EE016F10639F0F8016191AB
:1010C0008F01C1010E94AD05F6CF62E2B2CFCD9093
:1010D000DD90ED90FC90B701A601F7FE0BC06DE22C
:1010E000C1010E94100544275527BA014C195D091A
:1010F0006E097F09C1010E943A0585CD4D915D9130
:101100006D917C91F7CF8C916FE971E0811102C0F4
:1011100064EA71E0C1010E94A30575CDCF92DF9210
:10112000EF92FF920F931F93CF93DF93D82FC62F89
:101130000E949F016B017C018091B502811165C005
:1011400081E08093B5028093B4029FEF9093B30245
:101150001092B2029C0F9093B10280939002809102
:101160009002DD0FD82BD093900280918F028130B6
:1011700009F07FC010928F020E949F016B017C01D9
:10118000809190028093BB008091B7029091B80249
:10119000A091B902B091BA02892B8A2B8B2BA1F0B6
:1011A0000E949F010091B7021091B8022091B902EC
:1011B0003091BA026C197D098E099F09061717072D
:1011C0002807390708F442C08091BC0083FDD8CFBE
:1011D00085EC8093BC000E949F016B017C01809193
:1011E000B502813009F447C08091B2028C1710F427
:1011F000C091B202A1E9B2E0E9E6F2E080E08C172A
:1012000051F19D9191938F5FFACF8091B7029091A8
:10121000B802A091B902B091BA02892B8A2B8B2B0C
:1012200009F48ACF0E949F010091B7021091B80281
:101230002091B9023091BA026C197D098E099F097B
:10124000061717072807390708F076CF8091B602EE
:101250000E946A03C0E010928E02C0938D028C2F10
:10126000DF91CF911F910F91FF90EF90DF90CF9082
:10127000089585EEAECF8091B7029091B802A0910B
:10128000B902B091BA02892B8A2B8B2B09F4A7CF14
:101290000E949F010091B7021091B8022091B902FB
:1012A0003091BA026C197D098E099F09061717073C
:1012B0002807390708F093CFC9CFFF920F931F93E8
:1012C000CF93DF93C82F8B0186E70E9428016C2FF4
:1012D0008CE793E00E94C9040E948B03EC2FE695F3
:1012E000E77084E0E89FF0011124E356FC4F618130
:1012F0007281838194810E94C40186E70E94280143
:1013000060E08CE793E00E94C9040E948B03D82F11
:1013100063E086E70E948E088CE793E00E948204D7
:10132000F82E8CE793E00E948204C82F8CE793E0AC
:101330000E94820430E020E0D130C1F0D11119C008
:101340004C2F50E070E060E0762F652F542F44273B
:101350006F29482BF8014083518362837383C9014D
:10136000DF91CF911F910F91FF90089521E030E020
:10137000F6CF22E030E0F3CF0F931F93CF938C0191
:10138000C62F0E94F8046C2F6460C8010E94F80404
:101390006C2F6B7FC8010E94F80483EC90E00197EA
:1013A000F1F7CF911F910F9108950F931F93CF9352
:1013B000DF938C01D62FC42F607F642B0E94BC0961
:1013C00080E1D89FB00111246C2BC801DF91CF912F
:1013D0001F910F910C94BC09CF93DF93CDB7DEB76B
:1013E00028970FB6F894DEBF0FBECDBF98E0E6E0B9
:1013F000F1E0DE01119601900D929A95E1F790913E
:101400001304981708F48FEF90E0880F991F21E0DC
:1014100030E02C0F3D1F820F931FFC0160816E5F37
:10142000606840E08BE094E028960FB6F894DEBF49
:101430000FBECDBFDF91CF910C94D5092F923F9273
:101440004F925F926F927F928F929F92AF92BF92D4
:10145000CF92DF92EF92FF920F931F93CF93DF9380
:10146000CDB7DEB7E9970FB6F894DEBF0FBECDBF9C
:101470009AAB89AB89E00E9434018AE00E94340172
:101480008BE00E94340160E089E00E94530160E03B
:101490008AE00E94530160E08BE00E94530165E006
:1014A00070E080E090E00E94C40186E70E9428017D
:1014B0000E948B03811107C380919B0381116CC033
:1014C0000BE813E080EAE82E86E70E9428016E2DE3
:1014D0008CE793E00E94C9040E948B03C82E62E04F
:1014E00086E70E948E088CE793E00E948204D82E43
:1014F0008CE793E00E94820421E0C21609F497C2AF
:101500003D2C212CD101A82BCD01F8018193919381
:101510008F01E394E394FEEAEF12D6CF40918B0360
:1015200050918C03BA01672F772762956F701092E4
:101530009A0310929903CA019F7090938C03809331
:101540008B0330E020E090E080E0F901EE7FE5578A
:10155000FC4FA081E18120FF8BC28A27A8E0FC011B
:10156000880F991FF7FF02C000E39027A150B9F739
:101570002F5F3F4F2031310541F750938C0340934B
:101580008B03892F992782958F706817790709F047
:101590004EC281E080939B0380919C03880FBE0123
:1015A0006B5F7F4F80650E945D09892B09F03FC208
:1015B00080919C03880FBE016F5F7F4F80640E9403
:1015C0005D09892B09F033C24D815E816F81788579
:1015D000411551056105710509F429C289819A8176
:1015E000AB81BC818FA398A7A9A7BAA7892B8A2B07
:1015F0008B2B09F41CC28091950390919603B0E067
:10160000A0E0BA2FA92F982F88277A018B01E81A1A
:10161000F90A0A0B1B0BE98AFA8A0B8B1C8B609167
:1016200097037091980390E080E0A80197010E94D1
:10163000D91A07E10E942C1B49019A018401005329
:10164000184F2F4F3F4F09871A872B873C8769898F
:101650007A898B899C899B01AC010E94D91AE98403
:10166000FA840B851C85A0EDEA16A7E0FA060105B1
:1016700011050CF001C2B3E0AB2EB12CC12CD12C62
:10168000E12CF12C00E010E00E94811A01E20E949E
:101690002C1B2DA33EA34BA75CA76DA77EA78FA7EE
:1016A00098ABE984FA840B851C85110FEE08FE2C9B
:1016B0008701ED86FE860F87188B29853A854B8535
:1016C0005C856D85762F862F962F205D37404109EA
:1016D00051096109710981099109322E432E542E55
:1016E000652E762E872E982E292E9DE3A92EE12C8D
:1016F000F12C00E010E0232D342D452D562D672DC3
:10170000782D892D922D0E94811AA32CB42CC52CE2
:10171000D62CE72CF82C092D122D0E94811A04E0FA
:101720000E942C1B2D8B3E8B4F8B588F698F7A8F8D
:101730008B8F9C8F2DE1A22EB12CC12CD12CE12CB2
:10174000F12C00E010E0232D342D452D562D672D72
:10175000782D892D922D0E94811AA32CB42CC52C92
:10176000D62CE72CF82C092D122D0E94811A04E0AA
:101770000E942C1B2D8F3E8F4F8F58A369A37AA3F5
:101780008BA39CA309851A852B853C8504321A4FAF
:101790002F4F3F4F0CF06EC029853A854B855C85F5
:1017A0006D85762F862F962F24523A4F4F4F5F4FDD
:1017B0006F4F7F4F8F4F9F4F322E432E542E652EEB
:1017C000762E872E982E292EF1E1AF2EB12CC12C2A
:1017D000D12CE12CF12C00E010E00E94811AA32C06
:1017E000B42CC52CD62CE72CF82C092D122D0E94D8
:1017F000811AAD88BE88CF88D88CE98CFA8C0B8D85
:101800001C8D0E94491B2D8B3E8B4F8B588F698FEF
:101810007A8F8B8F9C8FA9E0AA2EB12CC12CD12C52
:10182000E12CF12C00E010E0232D342D452D562D18
:10183000672D782D892D922D0E94811AA32CB42C0E
:10184000C52CD62CE72CF82C092D122D0E94811ABC
:10185000AD8CBE8CCF8CD8A0E9A0FAA00BA11CA1A6
:101860000E94491B2D8F3E8F4F8F58A369A37AA3E7
:101870008BA39CA3609193037091940390E080E00C
:1018800029893A894B895C890E94D91A06E00E940D
:101890002C1B39014A01B62FA72FF82FE92FA09052
:1018A0008F03B0909003950140E050E060E070E05D
:1018B00080E090E001E10E94131B59016A017B0165
:1018C0008C019301A4016B2F7A2F8F2F9E2F0E94E2
:1018D000491B2D873BAB4CAB5DAB6EAB7FAB88AF91
:1018E00099AF609191037091920390E080E0298913
:1018F0003A894B895C890E94D91A07E00E942C1B07
:1019000039014A01B62FA72FF82FE92FA0908D0398
:10191000B0908E03950140E050E060E070E080E020
:1019200090E000E10E94131B59016A017B018C01C8
:101930009301A4016B2F7A2F8F2F9E2F0E94491B9A
:1019400049016A017B018C0169857A858B859C85BB
:101950000E9481172B013C012DA13EA14BA55CA546
:101960006DA57EA58FA598A90E94F2199B01AC01D7
:10197000C301B2010E94E41820E030E048EC52E4D8
:101980000E9451196987798B8DA39EA39401A601AA
:10199000B701C801AD8CBE8CCF8CD8A0E9A0FAA04D
:1019A0000BA11CA10E94521BEFA0F8A409A51AA527
:1019B00057016801E12CF12C00E010E00E94811A2F
:1019C00005E10E942C1B522E632E4A01B62FA72F31
:1019D000F82FE92F2D853BA94CA95DA96EA97FA9F8
:1019E00088AD99ADAD88BE88CF88D88CE98CFA8C4B
:1019F0000B8D1C8D0E94521B59016A017B018C01C9
:101A0000252D362DA4016B2F7A2F8F2F9E2F0E940C
:101A1000521B0FE00E942C1B0E94F21920E030E0C4
:101A200048EC52E40E945119F62E672E4C0109A988
:101A30001AA9012B09F451C06F2D762DC401E99626
:101A40000FB6F894DEBF0FBECDBFDF91CF911F91CF
:101A50000F91FF90EF90DF90CF90BF90AF909F904D
:101A60008F907F906F905F904F903F902F90089550
:101A7000512C8E27952572CDE5E0AE2EB12CC12CD0
:101A8000D12CE12CF12C00E010E00E94811A06E23A
:101A90000E942C1B2DA33EA34BA75CA76DA77EA77E
:101AA0008FA798AB1D8E1E8E1F8E18A219A21AA288
:101AB0001BA21CA21D8A1E8A1F8A188E198E1A8EBE
:101AC0001B8E1C8ED7CE80E00E94EC096AEA71E082
:101AD0008BE094E00E949405AFCFF98469888DA0D3
:101AE0009EA0AACF40E061E08BE094E00E94D5097F
:101AF0008BE39FE10197F1F7089541E00E94D5093A
:101B000081E090E008950F931F93CF93DF93EC0152
:101B100088819981009759F02A813B8126173707E0
:101B200030F081E0DF91CF911F910F9108958B01EB
:101B30006F5F7F4F0E94861C009759F099838883BE
:101B40001B830A832C813D81232B59F7FC011082D2
:101B5000E8CF80E0E7CFEF92FF920F931F93CF93F0
:101B6000DF936115710541F480E0DF91CF911F9102
:101B70000F91FF90EF90089541155105B1F07B0151
:101B8000EC010C811D81040F151FB8010E94830D0B
:101B9000882351F3288139818C819D81B701820F7F
:101BA000931F0E94551D1D830C8381E0DECFCF93D0
:101BB000DF93EC0188819981009711F00E94FD1B51
:101BC000198218821D821C821B821A82DF91CF919A
:101BD0000895CF93DF93EC01FB0101900020E9F71A
:101BE0003197AF01461B570B0E94AB0D811103C00B
:101BF000CE010E94D70DCE01DF91CF910895CF93F2
:101C0000DF93EC01FB0144815581608171810E9469
:101C1000AB0D811103C0CE010E94D70DCE01DF9123
:101C2000CF910895EF92FF920F931F93CF93DF937D
:101C3000EC017B018A01BA010E94830D81110BC066
:101C4000CE010E94D70DCE01DF91CF911F910F9150
:101C5000FF90EF9008951D830C83B70188819981CF
:101C60000E94551DF0CFEF92FF920F931F93CF93D9
:101C7000DF93CDB7DEB7A1970FB6F894DEBF0FBEE6
:101C8000CDBF7C01CB01BA01F70111821082138212
:101C90001282158214828E010F5F1F4F22E044E0F2
:101CA0000E9425150097C9F0FC0101900020E9F77A
:101CB0003197AF01481B590BBC01C7010E94120E9E
:101CC000A1960FB6F894DEBF0FBECDBFDF91CF91C6
:101CD0001F910F91FF90EF900895C7010E94D70DBB
:101CE000EFCFCF93DF93EC01FB018617970749F005
:101CF000608171816115710541F0448155810E94B7
:101D0000120ECE01DF91CF9108950E94D70DF9CF29
:101D1000FC01118210821382128215821482FB014F
:101D200001900020E9F73197AF01461B570B0C9447
:101D3000120EFC0180819181009711F00C94FD1B23
:101D4000089585ED8093BC008091B7029091B80210
:101D5000A091B902B091BA020796A11DB11D23E06E
:101D6000B695A795979587952A95D1F72091BC00B0
:101D700024FD03C01092B50208954091B70250911E
:101D8000B8026091B9027091BA02452B462B472BDD
:101D900069F30097A105B10541F02AE22A95F1F710
:101DA00000C00197A109B109E1CF8091B6020C945E
:101DB0006A03CF92DF92EF92FF920F931F93CF931C
:101DC000DF93FC018481982F9F7739F480788062BB
:101DD00084831182108213821282848185FD0BC05C
:101DE00080E090E0DF91CF911F910F91FF90EF90F5
:101DF000DF90CF9008956115710591F3EA017B01A1
:101E00006F01008111810115110589F1D801169624
:101E10006D917C91C7010E944C1D892B31F1C80145
:101E20000E9486058C01EFCF3897FD83EC833097B5
:101E3000B9F2E601AA81BB81109791F0CF018A1B0C
:101E40009B0B23E0959587952A95E1F715968C9342
:101E5000FB83EA8315821482F782E682CF01C2CF28
:101E6000F983E883FB83EA83F5CFC801BBCFEC811C
:101E7000FD818A819B810896E817F907A8F681E021
:101E80008887AECF1F920F920FB60F9211242F9317
:101E90003F938F939F93AF93BF93809161029091F3
:101EA0006202A0916302B09164023091600223E06B
:101EB000230F2D3758F50196A11DB11D2093600207
:101EC0008093610290936202A0936302B0936402D4
:101ED0008091650290916602A0916702B0916802BC
:101EE0000196A11DB11D8093650290936602A09397
:101EF0006702B0936802BF91AF919F918F913F911C
:101F00002F910F900FBE0F901F90189526E8230F6A
:101F10000296A11DB11DD2CF1F920F920FB60F9244
:101F200011242F933F934F935F936F937F938F93DE
:101F30009F93AF93BF93EF93FF938FED92E00E9437
:101F40007E02FF91EF91BF91AF919F918F917F9111
:101F50006F915F914F913F912F910F900FBE0F9016
:101F60001F9018951F920F920FB60F9211242F9366
:101F70008F939F93EF93FF93E091EF02F091F00224
:101F80008081E091F502F091F60282FD1BC0908104
:101F90008091F8028F5F8F732091F902821741F0D0
:101FA000E091F802F0E0E152FD4F958F8093F80246
:101FB000FF91EF919F918F912F910F900FBE0F90F6
:101FC0001F9018958081F4CF1F920F920FB60F9239
:101FD00011242F933F934F935F936F937F938F932E
:101FE0009F93AF93BF93EF93FF938091B900887F46
:101FF000803609F44AC0F0F5883209F4A7C018F514
:10200000803109F49BC0B8F4882309F4F9C0883002
:1020100009F494C0FF91EF91BF91AF919F918F917F
:102020007F916F915F914F913F912F910F900FBED4
:102030000F901F901895883109F488C0803251F7AD
:102040008093B30214C0803409F49DC040F48033FF
:10205000B9F38833F9F68093B30285ECB0C08035CC
:1020600009F485C0883509F496C0883499F60E9431
:10207000A10ED0CF883909F48CC038F5883729F003
:1020800050F4883611F0803729F683E08093B5024A
:1020900010925F0257C0883809F47BC0803919F06C
:1020A000803809F0B7CF80915F02803208F071C0AC
:1020B000E0915F0281E08E0F80935F028091BB0010
:1020C000F0E0E15CFD4F80833DC0803B39F0E0F4FF
:1020D000803A09F479C0883A09F09CCF84E0809373
:1020E000B50210923E0210923D02E0918B02F091F7
:1020F0008C02099580913D0281110FC081E080938F
:102100003D0210921D0209C0803C09F4A6CF883C14
:1021100009F4A3CF883B09F07DCFE0913E0281E036
:102120008E0F80933E02F0E0E35EFD4F808180934E
:10213000BB0090913E0280913D0229C080919002A7
:102140008093BB0085EC8093BC0064CF9091B20279
:102150008091B102981758F5E091B20281E08E0F9C
:102160008093B202F0E0EF56FD4F8081E9CFE0911D
:10217000B20281E08E0F8093B2028091BB00F0E04A
:10218000EF56FD4F80839091B2028091B102981773
:10219000C8F285E8D8CFE091B20281E08E0F80933B
:1021A000B2028091BB00F0E0EF56FD4F808380913A
:1021B000B40281115CCF81E080938F0284EA809326
:1021C000BC001092B50226CF85EC8093BC00109223
:1021D000B50280915F02803230F4E0915F02F0E05E
:1021E000E15CFD4F108260915F0270E0E091890236
:1021F000F0918A028FE392E0099510925F020ACF74
:102200001092B30234CFCF93DF93EFEDF2E013825D
:10221000128288EE93E0A0E0B0E084839583A683E9
:10222000B78326E531E03183208325EC30E0358724
:10223000248724EC30E03787268720EC30E0318B90
:10224000208B21EC30E0338B228B22EC30E0358B7D
:10225000248B26EC30E0378B268B118E128E138E5A
:10226000148EECE7F3E01382128284839583A683B5
:10227000B78388E691E091838083EBE0F4E01382FA
:1022800012828AE791E09183808387E2848380E1F0
:10229000818782E0828713861092890310928803D7
:1022A000CAE8D3E0198A88E1EEE0F1E0AEE9B3E0F4
:1022B00001900D928A95E1F788E1E6E2F1E0AEEB5C
:1022C000B3E001900D928A95E1F780EA90E0A0E0FA
:1022D000B0E08EA79FA7A8ABB9AB81E090E09DA727
:1022E0008CA71AAA1BAA87E78093D60384E1EEE3A2
:1022F000F1E0A7EDB3E001900D928A95E1F710921D
:10230000FB031092FC03DF91CF910895CF93DF93ED
:10231000CDB7DEB7C959D1090FB6F894DEBF0FBEED
:10232000CDBF789484B5826084BD84B5816084BD5E
:1023300085B5826085BD85B5816085BD80916E0063
:10234000816080936E001092810080918100826094
:1023500080938100809181008160809381008091D1
:1023600080008160809380008091B10084608093C0
:10237000B1008091B00081608093B00080917A00BC
:10238000846080937A0080917A00826080937A00E2
:1023900080917A00816080937A0080917A008068D1
:1023A00080937A001092C100E091EF02F091F00268
:1023B00082E08083E091EB02F091EC021082E091E8
:1023C000ED02F091EE028FEC80831092F702E09123
:1023D000F302F091F40286E08083E091F102F09143
:1023E000F202808180618083E091F102F091F2023B
:1023F000808188608083E091F102F091F202808117
:1024000080688083E091F102F091F20280818F7DFB
:10241000808389E00E9434018AE00E9434018BE0CD
:102420000E94340161E089E00E94530161E08AE08A
:102430000E94530161E08BE00E9453010E9453030C
:102440000E9453030E9453030E9453030E945303AC
:102450000E9453031092100480911504823018F0EA
:1024600098E0909310048093130462E370E080E09E
:1024700090E00E94C401609116048BE094E00E94F9
:10248000F80468EE73E080E090E00E94C40160E32D
:102490008BE094E00E94BC090BE416E4C8010197AC
:1024A000F1F760E38BE094E00E94BC09C80101975A
:1024B000F1F760E38BE094E00E94BC0983E592E0D1
:1024C0000197F1F760E28BE094E00E94BC09609113
:1024D0001004606240E08BE094E00E94D50984E043
:1024E0008093110440E06CE08BE094E00E94D509F9
:1024F0000E94720D82E08093120440E066E08BE05F
:1025000094E00E94D50940E062E08BE094E00E94F4
:10251000D5098BE39FE10197F1F788E080931604DA
:1025200060E08BE094E00E94F8046DEB71E08BE0DA
:1025300094E00E9494056FEC71E08BE094E00E94BF
:1025400094050E94720D1E012FE0220E311C3A826A
:1025500029823C822B8283E790E08C0F9D1F9E8313
:102560008D8398878F8319861E8690E080E00E9475
:102570001E0A4B015C0181E090E00E941E0ACF56CA
:10258000DF4F688379838A839B83C159D04089E078
:102590000E9434018AE00E9434018BE00E943401E1
:1025A00060E089E00E94530160E08AE00E945301EC
:1025B00060E08BE00E94530165E070E080E090E015
:1025C0000E94C40180E40E9428010E948B038111B3
:1025D00032C2109289031092880380E40E9428017D
:1025E00063EF8CE793E00E94C9040E948B0362E3CF
:1025F00070E080E090E00E94C40163E080E40E940B
:102600008E088CE793E00E948204E4968FAFE497F3
:102610008CE793E00E948204E5968FAFE5978CE704
:1026200093E00E948204CB56DF4F8883C559D04087
:10263000E6968FAFE697E5968EAD9FADE597982726
:1026400089279827B0E0A0E0BA2FA92F982F8827D4
:10265000E0E1F0E040E050E86FEF70E0C12C30E8DE
:10266000D32E38E9E32EF12C00E010E020E830E032
:1026700028013901482259226A227B22452846280E
:10268000472851F02601370144225522662277223D
:1026900084259525A625B725369527951795079561
:1026A0007695679557954795F694E794D794C79490
:1026B0003197F1F6CB56DF4F2881C559D040422FD4
:1026C00050E070E060E0481759076A077B0709F09F
:1026D0004DC080E40E94280165EF8CE793E00E94E2
:1026E000C9040E948B0362E370E080E090E00E94E6
:1026F000C40163E080E40E948E088CE793E00E94AE
:102700008204E4968FAFE4978CE793E00E94820402
:10271000E5968FAFE5978CE793E00E9482040E94D4
:102720008B03E5966EAD7FADE59776276727762715
:1027300090E080E00E947F1720E030E04AEF52E412
:102740000E94E01720E030E040E857E30E94E017E5
:1027500020E030E040EC50E40E94E418CA56DF4F1D
:10276000688379838A839B83C659D0400E94720D07
:10277000B501A401CE018D589F4F0E94330E65EE26
:1027800071E0CE0187589F4F0E94880EBE016D58A0
:102790007F4FCE0187589F4F0E94FF0D69EE71E079
:1027A0000E94E90DC557DF4F19821882CB58D040DF
:1027B000C357DF4F19821882CD58D040C157DF4F21
:1027C00019821882CF58D040BC01CE0185579F4F47
:1027D0000E94710ECE0187589F4F0E94990ECE0124
:1027E0008D589F4F0E94990E80E00E94EC09CE0107
:1027F00085579F4F0E942402CA56DF4F4881598156
:102800006A817B81C659D040CE018D589F4F0E946E
:10281000330E6CEE71E0CE0187589F4F0E94880EF8
:10282000BE016D587F4FCE0187589F4F0E94FF0D0C
:1028300060EF71E00E94E90DCB57DF4F19821882DB
:10284000C558D040C957DF4F19821882C758D040A9
:10285000C757DF4F19821882C958D040BC01CE013A
:102860008B579F4F0E94710ECE0187589F4F0E9439
:10287000990ECE018D589F4F0E94990E81E00E94C3
:10288000EC09CE018B579F4F0E94240260E177E252
:1028900080E090E00E94C401CF56DF4F488159810B
:1028A0006A817B81C159D040CE018D589F4F0E94D3
:1028B000330E65EF71E0CE0187589F4F0E94880E5E
:1028C000BE016D587F4FCE0187589F4F0E94FF0D6C
:1028D00069EF71E00E94E90DC158DF4F198218823B
:1028E000CF57D040CF57DF4F19821882C158D04000
:1028F000CD57DF4F19821882C358D040BC01CE019A
:1029000081589F4F0E94710ECE0187589F4F0E94A1
:10291000990ECE018D589F4F0E94990E81E00E9422
:10292000EC09CE0181589F4F0E942402CE018158AC
:102930009F4F0E94990ECE018B579F4F0E94990E78
:10294000CE0185579F4F0E94990EAE014F5F5F4F9A
:102950006EEF71E0CE010A960E94D90EFC01892B20
:1029600041F0948190789C60948380829182A282CD
:10297000B382AE014F5F5F4F6AE072E0CE010A960C
:102980000E94D90EFC01892B81F0948190789C6083
:102990009483CA56DF4F88819981AA81BB81C65929
:1029A000D04080839183A283B383AE014F5F5F4F9A
:1029B00063E172E0CE010A960E94D90EFC01892BD8
:1029C00081F0948190789C609483CF56DF4F88810A
:1029D0009981AA81BB81C159D04080839183A28310
:1029E000B383AFEDB2E0E596BFAFAEAFE597E79644
:1029F0001FAE1EAEE797BE016D587F4FCE010A96FF
:102A00000E94CD056FEC71E08FED92E00E9494057D
:102A100060ED77E080E090E00E94C40180E090E00B
:102A2000892B09F494CD0E946A02882309F48FCD82
:102A30000E9400008CCD80E00E94EC0962ED71E004
:102A40008BE094E00E94940591CEEF920F931F9338
:102A5000CF93DF93E80134E047FD34E1042E000C0E
:102A6000550B57FF03C0519541955109E32E022F95
:102A7000242FAE010E944315CE01DF91CF911F910B
:102A80000F91EF900895A9E0B0E0E9E4F5E10C942E
:102A9000A4186A01F22EB02E102FFBE3AF2EA01661
:102AA00008F41BE31F5F012F27E0AE014F5F5F4F6C
:102AB0000E94A216BC018981982F9970913009F467
:102AC0003FC09BE2E1FC04C09E2D9170E0FC3AC047
:102AD0005E2D5071E82FE87083FF46C084E09111AD
:102AE00001C083E0EF2DE81B8F1508F0E0E0D60170
:102AF0008E2F20E2552351F1992329F0D6019C9382
:102B0000C60101966C0196012D5F3F4FE2FE24C085
:102B10008EE4D6018C9391E411969C9311971296B2
:102B20008C93D9018E2F90E281111BC0E20FF32FFD
:102B3000F11D10828EEF9FEF2996ECE00C94C018E7
:102B40009DE2C6CF90E2C4CF2D9381508111FCCF7E
:102B5000CE0ED11CE0E0D0CF8EE6D6018C9391E66C
:102B6000DBCF9D938150E0CF482F447082FF3DC062
:102B700084E0911101C083E08F1510F4EF2DE81B64
:102B8000D6018E2F20E2552309F1992329F0D60191
:102B90009C93C60101966C0196012D5F3F4FE2FEAA
:102BA0001BC089E4D6018C938EE411968C93119707
:102BB00086E412968C93D9018E2F90E2882309F433
:102BC000B5CF9D938150FACF2D9381508111FCCFC9
:102BD000CE0ED11CE0E0D9CF89E6D6018C938EE6EB
:102BE00011968C93119786E6E4CF9B0177FF02C084
:102BF00030E020E0A1E0B0E0911102C0B0E0A0E040
:102C0000F9013196AE0FBF1F8B2C912CBB2009F41C
:102C100061C05401EFEFAE1ABE0AAA0DBB1DFA1631
:102C20001B0619F014F04F2D4A1B511188C0E3FC0C
:102C300059C07601A42FB0E2A1114FC0C40ED11C1F
:102C4000992309F45BC040E0D6011196F601908308
:102C50006D01552309F448C0012F060F9A81582FA2
:102C6000507184FF03C0913309F4015010160CF029
:102C700047C0093008F008E0EEE2FE2E5B01A01A22
:102C8000B10885019194819491082F3F320729F46E
:102C9000D601FC92F60131966F016217730794F129
:102CA000021713077CF5DB01A21BB30BAA24A39424
:102CB000B12CAC0EBD1EAA0DBB1D11968C912150DE
:102CC0003109D601119628153905F4F0F6018083F3
:102CD0006D01DBCFB12CA12CA0CFF701B1937F0107
:102CE000A150AACF9111B0CFD601942F50E302C0CA
:102CF0005D9391509111FCCFC40ED11C40E0ACCF3C
:102D000001E0BACF80E3DBCF6217730731F496336B
:102D100088F4953311F4552369F0F6018083FD01A1
:102D2000842F90E2811108C0A40FB11D1C9290E085
:102D300080E002CF81E3F1CF91938150F3CF9111E5
:102D400083CF8ACF283008F027E03327DA01990FA4
:102D5000311D87FD916000966105710539F432607F
:102D60002E5F3D9330E32A95E1F708959F3F30F0C1
:102D700080387105610509F03C5F3C5F3D939130FF
:102D800008F08068911DDF93CF931F930F93FF92FC
:102D9000EF92192F987F9695E92F96959695E90FC2
:102DA000FF27EE53FF4F99273327EE24FF24A70177
:102DB000E70105900894079428F4360FE71EF81EE3
:102DC000491F511D660F771F881F991F0694A1F791
:102DD0000590079428F4E70EF81E491F561FC11DE1
:102DE000770F881F991F661F0694A1F70590079417
:102DF00028F4F80E491F561FC71FD11D880F991FB1
:102E0000661F771F0694A1F70590079420F4490FD9
:102E1000561FC71FD81F990F661F771F881F06945C
:102E2000A9F784911095177041F0D695C7955795DD
:102E30004795F794E7941A95C1F7E8E6F0E06894AF
:102E40001590159135916591959105907FE2739557
:102E5000E118F10A430B560BC90BD009C0F7E10C7E
:102E6000F11E431F561FC91FD01D7EF4703311F48D
:102E70008A95E6CFE894015030F0080F0AF4002755
:102E8000021708F4202F2395022F7A3328F079E3D4
:102E90007D932A95E9F710C07D932A9589F60694CB
:102EA00097956795379517951794E118F10A430B95
:102EB000560BC90BD00998F023957E9173957A3300
:102EC00008F070E37C932013B8F77E9170617D93D6
:102ED00030F0839571E37D9370E32A95E1F7112437
:102EE000EF90FF900F911F91CF91DF91992787FD70
:102EF000909508950E94BC1708F481E00895E89425
:102F000009C097FB3EF490958095709561957F4F31
:102F10008F4F9F4F9923A9F0F92F96E9BB279395DF
:102F2000F695879577956795B795F111F8CFFAF4EF
:102F3000BB0F11F460FF1BC06F5F7F4F8F4F9F4F20
:102F400016C0882311F096E911C0772321F09EE87E
:102F5000872F762F05C0662371F096E8862F70E0E4
:102F600060E02AF09A95660F771F881FDAF7880FBE
:102F70009695879597F90895990F0008550FAA0B14
:102F8000E0E8FEEF16161706E807F907C0F012167C
:102F90001306E407F50798F0621B730B840B950B7F
:102FA00039F40A2661F0232B242B252B21F40895D4
:102FB0000A2609F4A140A6958FEF811D811D089571
:102FC0000E94F3170C9464180E94561838F00E945F
:102FD0005D1820F0952311F00C944D180C945318A3
:102FE00011240C9498180E94751870F3959FC1F3E2
:102FF000950F50E0551F629FF001729FBB27F00DA7
:10300000B11D639FAA27F00DB11DAA1F649F6627FB
:10301000B00DA11D661F829F2227B00DA11D621F4A
:10302000739FB00DA11D621F839FA00D611D221F04
:10303000749F3327A00D611D231F849F600D211DE8
:10304000822F762F6A2F11249F5750409AF0F1F06B
:1030500088234AF0EE0FFF1FBB1F661F771F881FD4
:1030600091505040A9F79E3F510580F00C944D18A7
:103070000C9498185F3FE4F3983ED4F386957795C7
:103080006795B795F795E7959F5FC1F7FE2B880F7A
:10309000911D9695879597F9089597F99F6780E810
:1030A00070E060E008959FEF80EC089500240A949A
:1030B0001616170618060906089500240A94121613
:1030C0001306140605060895092E0394000C11F446
:1030D000882352F0BB0F40F4BF2B11F460FF04C0F3
:1030E0006F5F7F4F8F4F9F4F089557FD9058440F4C
:1030F000551F59F05F3F71F04795880F97FB991F57
:1031000061F09F3F79F08795089512161306140613
:10311000551FF2CF4695F1DF08C0161617061806A0
:10312000991FF1CF86957105610508940895E8947B
:10313000BB2766277727CB0197F908952F923F92F7
:103140004F925F926F927F928F929F92AF92BF92B7
:10315000CF92DF92EF92FF920F931F93CF93DF9363
:10316000CDB7DEB7CA1BDB0B0FB6F894DEBF0FBEC0
:10317000CDBF09942A88398848885F846E847D840D
:103180008C849B84AA84B984C884DF80EE80FD800F
:103190000C811B81AA81B981CE0FD11D0FB6F89485
:1031A000DEBF0FBECDBFED010895A29FB001B39F5A
:1031B000C001A39F700D811D1124911DB29F700D40
:1031C000811D1124911D08955058BB27AA270E94E4
:1031D000FC180C9464180E94561838F00E945D1870
:1031E00020F039F49F3F19F426F40C9453180EF490
:1031F000E095E7FB0C944D18E92F0E94751858F3E1
:10320000BA17620773078407950720F079F4A6F5CB
:103210000C9497180EF4E0950B2EBA2FA02D0B01ED
:10322000B90190010C01CA01A0011124FF27591B0B
:1032300099F0593F50F4503E68F11A16F040A22F11
:10324000232F342F4427585FF3CF46953795279582
:10325000A795F0405395C9F77EF41F16BA0B620B81
:10326000730B840BBAF09150A1F0FF0FBB1F661FC8
:10327000771F881FC2F70EC0BA0F621F731F841F0B
:1032800048F4879577956795B795F7959E3F08F031
:10329000B0CF9395880F08F09927EE0F97958795F3
:1032A00008950E9465190C9464180E945D1858F0E6
:1032B0000E94561840F029F45F3F29F00C944D18F5
:1032C00051110C9498180C9453180E94751868F3B7
:1032D0009923B1F3552391F3951B550BBB27AA27CF
:1032E00062177307840738F09F5F5F4F220F331F09
:1032F000441FAA1FA9F335D00E2E3AF0E0E832D0D1
:1033000091505040E695001CCAF72BD0FE2F29D0D3
:10331000660F771F881FBB1F261737074807AB07A5
:10332000B0E809F0BB0B802DBF01FF2793585F4F1A
:103330003AF09E3F510578F00C944D180C94981873
:103340005F3FE4F3983ED4F3869577956795B795FC
:10335000F7959F5FC9F7880F911D9695879597F907
:103360000895E1E0660F771F881FBB1F6217730780
:103370008407BA0720F0621B730B840BBA0BEE1F95
:1033800088F7E09508950E947D1888F09F5798F07F
:10339000B92F9927B751B0F0E1F0660F771F881F5A
:1033A000991F1AF0BA95C9F714C0B13091F00E9474
:1033B0009718B1E008950C949718672F782F8827F5
:1033C000B85F39F0B93FCCF3869577956795B3959B
:1033D000D9F73EF490958095709561957F4F8F4F0A
:1033E0009F4F089597FB16F40E94361A0C94F91912
:1033F000E894F92F96EBFF2381F0121613061406BA
:10340000440B9395F695879577956795579540402A
:10341000FF23B9F71BC099270895882351F49850CA
:10342000D2F7872B762F652F542F432F322F20E092
:10343000B1F3121613061406440B88233AF09A953A
:10344000440F551F661F771F881FCAF755234AF47C
:10345000440F551F11F460FF04C06F5F7F4F8F4F03
:103460009F4F880F9695879597F908959095809529
:103470007095609550954095309521953F4F4F4FF1
:103480005F4F6F4F7F4F8F4F9F4F08950E94BC1724
:1034900008F48FEF0895AA1BBB1B51E107C0AA1FB8
:1034A000BB1FA617B70710F0A61BB70B881F991FE5
:1034B0005A95A9F780959095BC01CD010895A1E298
:1034C0001A2EAA1BBB1BFD010DC0AA1FBB1FEE1F9E
:1034D000FF1FA217B307E407F50720F0A21BB30BE9
:1034E000E40BF50B661F771F881F991F1A9469F765
:1034F00060957095809590959B01AC01BD01CF01C1
:103500000895DF93CF931F930F939A9DF02D219FE2
:10351000F00D8B9DF00D8A9DE02DF10D039FF00DB8
:10352000029FE00DF11D4E9DE00DF11D5E9DF00D21
:103530004F9DF00D7F936F93BF92AF925F934F9328
:10354000D5010E94D5188B01AC01D7010E94D51876
:10355000EB01E80FF91FD6010E94D01A2F913F917D
:10356000D6010E94D518C60FD71FE81FF91FAF91CB
:10357000BF910E94D01A2F913F910E94D518C60F7B
:10358000D71FE81FF91FD6010E94D518E60FF71FB5
:103590009801BE01CF010F911F91CF91DF91089546
:1035A0000E94D518460F571FC81FD91F08F431961F
:1035B000089597FB57FF0C94E91A9F938F930E94ED
:1035C000E91A6E1B7F0BAF91BF918A0B9B0B08957D
:1035D000E894DF93CF93FC01DB010E94D5187F9321
:1035E0006F93E9019A01AC01BF93AF933F932F937F
:1035F000DF010E94D51826F46C1B7D0B820B930B08
:103600009E01EB01FC010E94D01AAF91BF912F9156
:103610003F910E94D01ABE01CF01F9012F913F9135
:10362000CF91DF910895002E083090F0982F872FCA
:10363000762F652F542F432F322F22270850F4CF97
:10364000220F331F441F551F661F771F881F991FA6
:103650000A95B2F7002D089597FD1094002E0830BA
:1036600098F00850232F342F452F562F672F782F8F
:10367000892F912DF4CF1594979587957795679518
:1036800057954795379527950A95AAF71124002D48
:1036900008952A0D3B1D4C1D5D1D6E1D7F1D801F55
:1036A000911F08952A193B094C095D096E097F098C
:1036B000800B910B0895EE0FFF1F0590F491E02D04
:1036C00009940F931F93CF93DF938230910510F4E9
:1036D00082E090E0E0911904F0911A0430E020E0DB
:1036E000B0E0A0E0309799F42115310509F44AC003
:1036F000281B390B24303105D8F58A819B8161154F
:10370000710589F1FB0193838283FE0111C0408121
:1037100051810281138148175907E0F04817590772
:1037200099F4109761F012960C93129713961C93CC
:103730003296CF01DF91CF911F910F9108950093A1
:10374000190410931A04F4CF2115310551F04217D2
:10375000530738F0A901DB019A01BD01DF01F8012F
:10376000C1CFEF01F9CF90931A0480931904CDCF04
:10377000FE01E20FF31F81939193225031093983A7
:103780002883D7CF2091170430911804232B41F4BC
:103790002091020130910301309318042093170403
:1037A00020910001309101012115310541F42DB71F
:1037B0003EB74091040150910501241B350BE09167
:1037C0001704F0911804E217F307A0F42E1B3F0B27
:1037D0002817390778F0AC014E5F5F4F2417350783
:1037E00048F04E0F5F1F50931804409317048193C5
:1037F00091939FCFF0E0E0E09CCFCF93DF930097D1
:10380000E9F0FC01329713821282A0911904B09161
:103810001A04ED0130E020E01097A1F420813181FD
:10382000820F931F2091170430911804281739072D
:1038300009F061C0F0931804E0931704DF91CF9171
:103840000895EA01CE17DF07E8F54A815B819E0102
:1038500041155105B1F7E901FB83EA83499159917B
:10386000C40FD51FEC17FD0761F48081918102968A
:10387000840F951FE90199838883828193819B83BB
:103880008A83F0E0E0E012968D919C911397009767
:10389000B9F52D913C911197CD010296820F931F9E
:1038A00020911704309118042817390739F63097FA
:1038B00051F510921A0410921904B0931804A093B1
:1038C0001704BCCFD383C28340815181840F951FDD
:1038D000C817D90761F44E5F5F4F88819981480FFF
:1038E000591F518340838A819B8193838283211551
:1038F000310509F0B0CFF0931A04E09319049ECF7C
:10390000FD01DC01C0CF13821282D7CFB0E0A0E06E
:10391000ECE8FCE10C94A0188C01009751F4CB0169
:103920000E94611B8C01C801CDB7DEB7E0E10C94A9
:10393000BC18FC01E60FF71F9C0122503109E21769
:10394000F30708F49DC0D901CD91DC911197C617FA
:10395000D70798F0C530D10530F3CE01049786170C
:10396000970708F3C61BD70B2297C193D1936D938A
:103970007C93CF010E94FD1BD6CF5B01AC1ABD0A20
:103980004C018C0E9D1EA0911904B0911A04512C6B
:10399000412CF12CE12C109731F580911704909176
:1039A00018048815990509F05CC04616570608F0FA
:1039B00058C08091000190910101009741F48DB7AA
:1039C0009EB74091040150910501841B950BE817A7
:1039D000F90708F055C0F0931804E0931704F901B3
:1039E00071836083A0CF8D919C91119712966C90FA
:1039F000129713967C901397A815B90559F56C0189
:103A000042E0C40ED11CCA14DB0420F1AC014A19F7
:103A10005B09DA011296159780F0628273825183F6
:103A20004083D9016D937C93E114F10471F0D701C7
:103A30001396FC93EE93129776CF22968C0F9D1FD0
:103A4000F90191838083F301EFCFF0931A04E0939F
:103A5000190469CF4816590608F42C017D01D301D9
:103A60009ACFCB010E94611B7C01009749F0AE0107
:103A7000B8010E94431DC8010E94FD1B870153CF5E
:103A800010E000E050CFFB01DC0102C001900D927C
:103A900041505040D8F70895FB01DC018D91019011
:103AA00080190110D9F3990B0895FB01DC010190F5
:103AB0000D920020E1F70895F894FFCF00001B0459
:103AC00080000000400014005400010000000200CB
:103AD00000000300000005000000090000001100C4
:103AE00000000100000002000000030000000500CB
:103AF000000009000000120000000000C0BF00002C
:103B0000803F000000C000008040000000C00000B6
:103B10000000A002F7012D02ED025E023C025002FD
:103B200000000000C9049C040D0572049504820481
:103B30007304000000007D0DF7010D050D032F2F0C
:103B400022225C5C6208660C6E0A720D7409005CCD
:103B50007530303030006E756C6C007472756500B5
:103B600066616C7365004E6170616B612073656E98
:103B70007A6F726A61203221005672656D656E73CC
:103B80006B6120706F7374616A61000D0A004E6191
:103B900070616B612073656E7A6F726A612031218A
:103BA00000543A2000204300483A20002025524883
:103BB00000503A2000206850610074656D70657295
:103BC00061747572650068756D69646974790070F7
:083BD0007265737375726500E4
:107E0000112484B714BE81FFF0D085E080938100F7
:107E100082E08093C00088E18093C10086E0809377
:107E2000C20080E18093C4008EE0C9D0259A86E02C
:107E300020E33CEF91E0309385002093840096BBD3
:107E4000B09BFECF1D9AA8958150A9F7CC24DD24C4
:107E500088248394B5E0AB2EA1E19A2EF3E0BF2EE7
:107E6000A2D0813461F49FD0082FAFD0023811F036
:107E7000013811F484E001C083E08DD089C08234E0
:107E800011F484E103C0853419F485E0A6D080C0E4
:107E9000853579F488D0E82EFF2485D0082F10E0AE
:107EA000102F00270E291F29000F111F8ED06801E7
:107EB0006FC0863521F484E090D080E0DECF843638
:107EC00009F040C070D06FD0082F6DD080E0C81688
:107ED00080E7D80618F4F601B7BEE895C0E0D1E017
:107EE00062D089930C17E1F7F0E0CF16F0E7DF06D8
:107EF00018F0F601B7BEE89568D007B600FCFDCFD4
:107F0000A601A0E0B1E02C9130E011968C91119780
:107F100090E0982F8827822B932B1296FA010C0160
:107F200087BEE89511244E5F5F4FF1E0A038BF0790
:107F300051F7F601A7BEE89507B600FCFDCF97BE46
:107F4000E89526C08437B1F42ED02DD0F82E2BD052
:107F50003CD0F601EF2C8F010F5F1F4F84911BD097
:107F6000EA94F801C1F70894C11CD11CFA94CF0C13
:107F7000D11C0EC0853739F428D08EE10CD085E9AC
:107F80000AD08FE07ACF813511F488E018D01DD067
:107F900080E101D065CF982F8091C00085FFFCCF94
:107FA0009093C60008958091C00087FFFCCF809118
:107FB000C00084FD01C0A8958091C6000895E0E648
:107FC000F0E098E1908380830895EDDF803219F02E
:107FD00088E0F5DFFFCF84E1DECF1F93182FE3DFCA
:107FE0001150E9F7F2DF1F91089580E0E8DFEE27F6
:047FF000FF270994CA
:027FFE00040479
:00000001FF
